:100000000C945C000C9496050C94C3050C9484002D
:100010000C9484000C9484000C9484000C94840050
:100020000C9484000C9484000C9484000C94840040
:100030000C9484000C9484000C9484000C94840030
:100040000C94F0050C9484000C9422080C94840009
:100050000C9484000C9484000C9484000C94840010
:100060000C9484000C948400000024272A000025AE
:10007000282B000023262904040404040404040299
:100080000202020202030303030303010204081035
:100090002040800102040810200102040810200002
:1000A0000000070002010000030406000000000039
:1000B00000000000F401820411241FBECFEFD4E041
:1000C000DEBFCDBF11E0A0E0B1E0E4EDF1E102C0A0
:1000D00005900D92A833B107D9F712E0A8E3B1E07B
:1000E00001C01D92A530B107E1F710E0C8EBD0E0E8
:1000F00004C02297FE010E94E408C43BD107C9F75F
:100100000E947B040C94E8080C940000FC0110820F
:100110008FEF81831382128282E2848386E9858352
:10012000178216820895EF92FF920F931F93CF9339
:10013000DF93EC019B0177FF03C020E030E005C0B6
:10014000653B710514F024EB30E02983EC806D8170
:1001500070E06E197109882777FD8095982F982F88
:10016000872F762F662730E040E050E00E945F083E
:1001700024EB30E040E050E00E94B308FF2400E0B0
:1001800010E0102F0F2DFE2CEE24E20EF31E041FA4
:10019000151FC801B70120E430E040E050E00E94A4
:1001A000B3083B832A83DF91CF911F910F91FF907A
:1001B000EF9008955F926F927F928F929F92AF928D
:1001C000BF92CF92DF92EF92FF920F931F93DF9334
:1001D000CF93CDB7DEB76DB67EB6ADB65EB60E9434
:1001E000600620913A0130913B0140913C015091D1
:1001F0003D01621773078407950750F02C5E3F4F4F
:100200004F4F5F4F621773078407950708F4AFC01D
:1002100060933A0170933B0180933C0190933D01C0
:10022000E0913801F0913901BB2408C082819381AB
:10023000892B09F0B3940680F781E02D3097B1F750
:10024000BB2009F494C08B2D90E0880F991F2DB727
:100250003EB7281B390B0FB6F8943EBF0FBE2DBF1B
:10026000CDB6DEB60894C11CD11CA0913801B09166
:10027000390120E013C012968D919C911397892B20
:1002800049F0E22FF0E0EE0FFF1FEC0DFD1DB183F2
:10029000A0832F5F16960D90BC91A02D109759F753
:1002A0002CC0812F90E07C01EE0CFF1CEC0CFD1C9F
:1002B000D7016D917C91FC013197EE0FFF1FEC0D82
:1002C000FD1D40815181DB0112962D913C911397C8
:1002D000DA0112968D919C9113972817390730F403
:1002E000D7014D935C937183608301E01F5F1B1501
:1002F000C0F2002311F410E011C011E000E0F7CFCC
:10030000E12FF0E0EE0FFF1FEC0DFD1D0190F081DD
:10031000E02D61E080810E9466071F5F1B1580F35E
:10032000F6B4EE2400E010E08F2C99241EC0EE2DD0
:10033000F0E0EE0FFF1FEC0DFD1D0190F081E02DB0
:1003400022813381280D391D86B58F1510F4005098
:100350001F4FF82EC8018F0D911D28173907A0F7E0
:1003600060E080810E946607E394EB1400F38A2D1D
:10037000952D9C010FB6F8943EBF0FBE2DBF0FB652
:10038000F8947EBE0FBE6DBECF91DF911F910F918D
:10039000FF90EF90DF90CF90BF90AF909F908F90A5
:1003A0007F906F905F9008950F931F938C01FC01D5
:1003B00060838FEF81831382128280913801909144
:1003C000390197838683109339010093380160E0E7
:1003D00080810E94660761E0F80180810E944807E1
:1003E00081E01F910F9108958EE391E00E948600B5
:1003F00086E491E00E9486008EE491E00E948600EF
:100400000895BC0186E491E00E9493000895BC0128
:100410008EE391E00E94930008956BE570E08EE317
:1004200091E00E9493006AE570E086E491E00E940A
:10043000930008950F931F938C010E940D0264EBAB
:1004400070E0601B710B8EE391E00E949300B80195
:1004500086E491E00E9493001F910F9108950F93FD
:100460001F938C010E940D02B8018EE391E00E945F
:10047000930064EB70E0601B710B86E491E00E94D6
:1004800093001F910F910895EF92FF920F931F9386
:100490000E94DA008FE691E00E949004882309F41C
:1004A000E1C08FE691E00E948D0480936201482FA5
:1004B00050E09A01207F307080915801909159014D
:1004C0002817390709F0CEC09A012F7030702730F5
:1004D000310509F492C028303105D4F423303105B8
:1004E00009F459C02430310554F421303105D9F1D3
:1004F000223031050CF041C0232B59F1B3C0253017
:10050000310509F46DC0263031050CF074C051C0BE
:100510002B30310509F483C02C3031054CF42930DF
:10052000310509F470C02A3031050CF070C069C083
:100530002D30310509F483C02D3031050CF477C01E
:100540002E30310509F47DC02F30310509F08AC005
:100550007EC060E080912B010E94660784EB90E0F2
:100560000E941A027FC060E080912B010E94660702
:1005700084EB90E00E942F0275C060E080912B0117
:100580000E94660780E090E00E94070280E090E011
:100590000E94010241C060E080912B010E94660729
:1005A00084EB90E00E94010284EB90E00E9407023D
:1005B00059C084E690E090936C0180936B0181E0D8
:1005C00090E090936E0180936D010E9460066093AD
:1005D0006701709368018093690190936A0142C03A
:1005E00010926E0110926D0160E070E080911D012B
:1005F0000E94F00637C061E001C060E080911B01FD
:1006000023C061E001C060E0809129011DC060E06D
:1006100080912B010E94660764EB70E01FC060E0D0
:1006200080912B010E94660760E070E017C061E0D6
:1006300080912B010E9466070E940D0213C061E0A9
:1006400001C060E080911F010E9466070BC060E05E
:1006500080912B010E9466076DE570E08EE491E0C9
:100660000E9493000E9460069B01AC0160936301AD
:1006700070936401809365019093660180916D0190
:1006800090916E01019709F053C08091670190919C
:100690006801A0916901B0916A01281B390B4A0BCE
:1006A0005B0B80916B0190916C01AA2797FDA0953F
:1006B000BA2F281739074A075B07A0F16FEF70E0E0
:1006C00080911D010E94F006E0906301F0906401AA
:1006D0000091650110916601809167019091680118
:1006E000A0916901B0916A01A8019701281B390BFB
:1006F0004A0B5B0B80916B0190916C01880F991FE5
:10070000AA2797FDA095BA2F281739074A075B0734
:1007100078F0E0926701F09268010093690110930C
:100720006A0106C060E070E080911D010E94F00641
:100730001F910F91FF90EF90089540E05BE460E01F
:1007400070E08FE691E00E94930464E670E080E040
:1007500090E00E946E0660E070E080911D010E94B2
:10076000F00660912D0170912E018EE391E00E94C0
:10077000D40160912F017091300186E491E00E94D4
:10078000D40160912101709122018EE491E00E94D8
:10079000D4010E940D026DE570E08EE491E00E94AC
:1007A000930061E080911B010E94480761E0809105
:1007B0001D010E94480761E080911F010E944807C7
:1007C00060E08EE00E94480760E08FE00E944807EA
:1007D00060E080E10E94480760E081E10E944807F4
:1007E00061E08EE00E94660761E08FE00E9466078C
:1007F00061E080E10E94660761E081E10E94660796
:10080000809156010E94D206815092403CF081E0D6
:1008100090E090935B0180935A0104C010925B01B9
:1008200010925A01809123010E94D2068150924079
:100830003CF082E090E090935D0180935C0104C005
:1008400010925D0110925C01809125010E94D206F8
:10085000815092403CF084E090E090935F0180935F
:100860005E0104C010925F0110925E018091270129
:100870000E94D206815092403CF088E090E0909334
:1008800061018093600104C01092610110926001C7
:1008900080915C0190915D0120915A0130915B0142
:1008A000820F931F20915E0130915F01820F931F91
:1008B0002091600130916101820F931F9093590143
:1008C0008093580160E071E08FE691E00E94980407
:1008D00060915801709159018FE691E00E94860560
:1008E00060E080911F010E94660761E080912B010A
:1008F0000E94660708950E9498060E949D030E9428
:100900004402FDCF86E391E09093700180936F01E4
:100910000895862F0E94EA0708950E94030808950B
:100920000E94F2070895CB01BA010E94B107089511
:100930000F931F93CF93DF938C01EB0109C0219696
:10094000D801ED91FC910190F081E02DC80109954D
:1009500068816623A1F7DF91CF911F910F910895D0
:100960000F931F938C01DC01ED91FC910190F081BC
:10097000E02D6DE00995D801ED91FC910190F08199
:10098000E02D6AE0C80109951F910F9108952F92FB
:100990003F924F925F926F927F928F929F92AF920F
:1009A000BF92CF92DF92EF92FF920F931F93DF934C
:1009B000CF93CDB7DEB7A0970FB6F894DEBF0FBECA
:1009C000CDBF1C016A017B0141155105610571050F
:1009D00049F4DC01ED91FC910190F081E02D60E3A0
:1009E000099554C0882499245401422E5524662424
:1009F000772401E010E00C0F1D1F080D191DC70121
:100A0000B601A30192010E949108F8016083089445
:100A1000811C911CA11CB11CC701B601A30192014C
:100A20000E949108C901DA016C017D01C114D10451
:100A3000E104F104F1F681E0E82EF12CEC0EFD1E4C
:100A4000E80CF91C3E010894611C711CD501C4011D
:100A50000197A109B1096C01C818D90814C0F601A1
:100A6000EE0DFF1D60816A3010F4605D01C0695CAD
:100A7000D101ED91FC910190F081E02DC10109952A
:100A80000894E108F1086E147F0449F7A0960FB6A8
:100A9000F894DEBF0FBECDBFCF91DF911F910F91B4
:100AA000FF90EF90DF90CF90BF90AF909F908F908E
:100AB0007F906F905F904F903F902F900895EF92AE
:100AC000FF920F931F93CF93DF93EC017A018B0179
:100AD00077FF0FC0E881F9810190F081E02D6DE290
:100AE000099510950095F094E094E11CF11C011D0E
:100AF000111D2AE0B801A701CE010E94C704DF91B1
:100B0000CF911F910F91FF90EF9008950F931F9336
:100B10008C01AB01662757FD6095762F0E945F051B
:100B2000C8010E94B0041F910F9108951F920F9267
:100B30000FB60F9211242F933F934F935F936F93B0
:100B40007F938F939F93AF93BF93EF93FF93809186
:100B5000710190917201892B29F0E0917101F0915E
:100B600072010995FF91EF91BF91AF919F918F9184
:100B70007F916F915F914F913F912F910F900FBE99
:100B80000F901F9018951F920F920FB60F9211247D
:100B90002F933F934F935F936F937F938F939F9385
:100BA000AF93BF93EF93FF93809173019091740182
:100BB000892B29F0E0917301F09174010995FF915F
:100BC000EF91BF91AF919F918F917F916F915F91C5
:100BD0004F913F912F910F900FBE0F901F9018953E
:100BE0001F920F920FB60F9211242F938F939F9302
:100BF000AF93BF938091750190917601A091770199
:100C0000B09178010196A11DB11D8093750190935B
:100C10007601A0937701B09378018091790190914A
:100C20007A01A0917B01B0917C018050904CAF4F34
:100C3000BF4F8093790190937A01A0937B01B09389
:100C40007C0127C08091790190917A01A0917B016C
:100C5000B0917C0180589E43A040B04080937901C0
:100C600090937A01A0937B01B0937C0180917D01E8
:100C700090917E01A0917F01B09180010196A11D0C
:100C8000B11D80937D0190937E01A0937F01B0936D
:100C900080018091790190917A01A0917B01B091BE
:100CA0007C0181589E43A040B04060F6BF91AF9157
:100CB0009F918F912F910F900FBE0F901F901895BD
:100CC0008FB7F89420917D0130917E0140917F0192
:100CD000509180018FBFB901CA010895EF92FF9230
:100CE0000F931F937B018C018FB7F89440917D0186
:100CF00050917E0160917F01709180018FBF2FB76D
:100D0000F89480917D0190917E01A0917F01B09136
:100D100080012FBF841B950BA60BB70BE816F906B5
:100D20000A071B0760F71F910F91FF90EF9008953E
:100D3000789484B5826084BD84B5816084BD85B5B6
:100D4000826085BD85B5816085BDEEE6F0E080817D
:100D500081608083E1E8F0E080818260808380812F
:100D600081608083E0E8F0E0808181608083E1EB56
:100D7000F0E0808184608083E0EBF0E0808181603E
:100D80008083EAE7F0E080818460808380818260F4
:100D900080838081816080838081806880831092DD
:100DA000C10008958F70909131019295990F990F1C
:100DB000907C982B90937C0080917A008064809343
:100DC0007A0080917A0086FDFCCF209178004091D6
:100DD0007900942F80E030E0282B392BC901089549
:100DE0001F93CF93DF93182FEB0161E00E94480718
:100DF000E12FF0E0E156FF4F8491833051F4809170
:100E00008000806880938000D0938900C093880020
:100E10003BC0843051F480918000806280938000D8
:100E2000D0938B00C0938A002FC0813039F4209773
:100E300029F184B5806884BDC7BD26C0823039F4ED
:100E40002097E1F084B5806284BDC8BD1DC08630A6
:100E500041F48091B00080688093B000C093B300EB
:100E600013C0873041F48091B00080628093B0005D
:100E7000C093B40009C0C038D10514F460E001C0CB
:100E800061E0812F0E946607DF91CF911F91089545
:100E9000282F30E0C90185579F4FFC0194912958B4
:100EA0003F4FF9018491882381F0E82FF0E0E85961
:100EB000FF4FE491F0E0662329F480819095892327
:100EC000808308958081892B80830895482F50E086
:100ED000CA0181569F4FFC012491CA0185579F4F3B
:100EE000FC01949149585F4FFA0134913323C1F1C9
:100EF000222331F1233021F4809180008F7705C0C7
:100F0000243031F4809180008F7D8093800018C060
:100F1000213019F484B58F7704C0223021F484B5D0
:100F20008F7D84BD0DC0263021F48091B0008F7775
:100F300005C0273029F48091B0008F7D8093B000E8
:100F4000E32FF0E0E359FF4FE491F0E0662329F44A
:100F5000808190958923808308958081892B808367
:100F60000895EF92FF920F931F937B018C0122E073
:100F700030E040E050E00E94B308205C3D4B404F21
:100F80005F4FCA01B901A80197010E94B308C901C6
:100F9000DA010197A109B109292F3A2F4B2F5527C3
:100FA00047FD5A950196A11DB11D2093C5008150A2
:100FB0008093C400E1ECF0E08081806180838081D7
:100FC000886080838081806880831F910F91FF906B
:100FD000EF900895982F8091C00085FFFCCF9093EB
:100FE000C6000895809181019091820180589F4FA1
:100FF0002091830130918401821B930B60E870E0A3
:101000000E947E080895409183015091840180914F
:101010008101909182018417950719F42FEF3FEF1A
:101020000FC0FA01EB57FE4F2081CA01019660E81C
:1010300070E00E947E08909384018093830130E0E9
:10104000C90108951F920F920FB60F9211242F938A
:101050003F934F935F936F937F938F939F93AF9340
:10106000BF93EF93FF934091C600E0918101F0910F
:101070008201CF01019660E870E00E947E089C0129
:1010800080918301909184012817390739F0EB573B
:10109000FE4F40833093820120938101FF91EF91B5
:1010A000BF91AF919F918F917F916F915F914F9180
:1010B0003F912F910F900FBE0F901F901895629F38
:1010C000D001739FF001829FE00DF11D649FE00D40
:1010D000F11D929FF00D839FF00D749FF00D659FA1
:1010E000F00D9927729FB00DE11DF91F639FB00DA0
:1010F000E11DF91FBD01CF011124089597FB092EB1
:1011000007260AD077FD04D049D006D000201AF473
:10111000709561957F4F0895F6F7909581959F4F53
:101120000895A1E21A2EAA1BBB1BFD010DC0AA1F28
:10113000BB1FEE1FFF1FA217B307E407F50720F040
:10114000A21BB30BE40BF50B661F771F881F991FBB
:101150001A9469F760957095809590959B01AC0104
:10116000BD01CF01089597FB092E05260ED057FD2E
:1011700004D0D7DF0AD0001C38F450954095309544
:1011800021953F4F4F4F5F4F0895F6F7909580950B
:10119000709561957F4F8F4F9F4F0895AA1BBB1B82
:1011A00051E107C0AA1FBB1FA617B70710F0A61B67
:1011B000B70B881F991F5A95A9F780959095BC0188
:1011C000CD010895EE0FFF1F0590F491E02D0994D5
:0411D000F894FFCFC1
:1011D400486F6C612C20736F7920656C20726F628C
:1011E4006F74206E756D65726F200008000B00042B
:1011F4000002000100020003000500070009000AC4
:08120400000100000000890454
:00000001FF
